:020000040000FA
:1000000000040020810A000015070000610A0000BA
:100010001F07000029070000330700000000000050
:10002000000000000000000000000000A50A000021
:100030003D070000000000004707000051070000D6
:100040005B070000650700006F07000079070000EC
:10005000830700008D07000097070000A10700003C
:10006000AB070000B5070000BF070000C90700008C
:10007000D3070000DD070000E7070000F1070000DC
:10008000FB070000050800000F0800001908000029
:10009000230800002D080000370800004108000078
:1000A0004B080000550800005F08000069080000C8
:1000B000730800007D080000870800009108000018
:1000C0009B080000A5080000AF080000B908000068
:1000D000C3080000CD080000D7080000E1080000B8
:1000E000EB080000F5080000FF0800000909000007
:1000F000130900001D090000270900003109000054
:100100003B0900001FB500F003F88DE80F001FBD8C
:1001100000F0ACBC40F6FC7108684FF01022401CA7
:1001200008D00868401C09D00868401C04D0086842
:1001300000F037BA9069F5E79069F9E7704770B554
:100140000B46010B184400F6FF70040B4FF0805073
:100150000022090303692403406943431D1B104621
:1001600000F048FA29462046BDE8704000F042BA47
:10017000F0B54FF6FF734FF4B4751A466E1E11E0DA
:10018000A94201D3344600E00C46091B30F8027B3B
:10019000641E3B441A44F9D19CB204EB134394B25D
:1001A00004EB12420029EBD198B200EB134002EBB2
:1001B000124140EA0140F0BDF34992B00446D1E952
:1001C0000001CDE91001FF224021684600F0F4FB58
:1001D00094E80F008DE80F00684610A902E004C8FB
:1001E00041F8042D8842FAD110216846FFF7C0FF7C
:1001F0001090AA208DF8440000F099F9FFF78AFFCB
:1002000040F6FC7420684FF01025401C0FD0206889
:1002100010226946803000F078F92068401C08D030
:100220002068082210A900F070F900F061F9A869AF
:10023000EEE7A869F5E74FF080500369406940F6A2
:10024000FC71434308684FF01022401C06D0086838
:1002500000F58050834203D2092070479069F7E788
:100260000868401C04D00868401C03D00020704778
:100270009069F9E70420704770B504460068C34DE3
:10028000072876D2DFE800F033041929631E250021
:10029000D4E9026564682946304600F062F92A46CE
:1002A0002146304600F031F9AA002146304600F0E0
:1002B00057FB002800D0032070BD00F009FC4FF46C
:1002C000805007E0201D00F040F90028F4D100F034
:1002D000FFFB60682860002070BD241D94E80700C3
:1002E000920000F03DFB0028F6D00E2070BDFFF715
:1002F000A2FF0028FAD1D4E901034FF0805100EBAE
:10030000830208694D69684382420ED840F6F8704E
:1003100005684FF010226D1C09D0056805EB8305B8
:100320000B6949694B439D4203D9092070BD55694A
:10033000F4E70168491C03D00068401C02D003E0C8
:100340005069FAE70F2070BD2046FFF735FFFFF731
:1003500072FF0028F7D1201D00F0F7F80028F2D135
:1003600060680028F0D100F0E2F8FFF7D3FE00F05B
:10037000BFF8072070BD10B50C46182802D0012028
:10038000086010BD2068FFF777FF206010BD41684E
:10039000054609B1012700E0002740F6F8742068FF
:1003A0004FF01026401C2BD02068AA68920000F065
:1003B000D7FA38B3A86881002068401C27D020688D
:1003C000FFF7BDFED7B12068401C22D026684FF051
:1003D0008050AC686D68016942695143A9420DD9EA
:1003E000016940694143A14208D92146304600F0E5
:1003F000B8F822462946304600F087F800F078F831
:100400007069D2E700F093F8FFF784FEF6E77069B1
:10041000D6E77669DBE740F6FC7420684FF01026DB
:10042000401C23D02068401C0CD02068401C1FD0EA
:100430002568206805F18005401C1BD027683879A5
:10044000AA2819D040F6F8700168491C42D001680A
:10045000491C45D00168491C3ED001680968491C07
:100460003ED00168491C39D000683EE0B069DAE747
:10047000B569DEE7B769E2E710212846FFF778FEA5
:100480003968814222D12068401C05D0D4F8001080
:1004900001F18002C03107E0B169F9E730B108CA63
:1004A00051F8040D984201D1012000E000208A4259
:1004B000F4D158B1286810B1042803D0FEE72846CB
:1004C000FFF765FF3149686808600EE0FFF722FE1C
:1004D00000F00EF87169BBE77169BFE7706904E06D
:1004E0004FF480500168491C01D000F0CBFAFEE7C0
:1004F000BFF34F8F26480168264A01F4E06111439B
:100500000160BFF34F8F00BFFDE72DE9F0411746B3
:100510000D460646002406E03046296800F054F8EF
:10052000641C2D1D361DBC42F6D3BDE8F08140F69B
:10053000FC700168491C04D0D0F800004FF48051D1
:10054000FDE54FF010208069F8E74FF080510A690F
:10055000496900684A43824201D810207047002050
:10056000704770B50C4605464FF4806608E0284693
:1005700000F017F8B44205D3A4F5806405F5805562
:10058000002CF4D170BD0000F40A0000000000202F
:100590000CED00E00400FA05144801680029FCD0C5
:1005A0007047134A0221116010490B68002BFCD0E0
:1005B0000F4B1B1D186008680028FCD0002010603D
:1005C00008680028FCD07047094B10B501221A605A
:1005D000064A1468002CFCD0016010680028FCD08A
:1005E0000020186010680028FCD010BD00E4014015
:1005F00004E5014070B50C46054600F073F810B9EB
:1006000000F07EF828B121462846BDE8704000F091
:1006100007B821462846BDE8704000F037B8000012
:100620007FB5002200920192029203920A0B000B06
:100630006946012302440AE0440900F01F0651F80C
:10064000245003FA06F6354341F82450401C8242F8
:10065000F2D80D490868009A10430860081D016827
:10066000019A1143016000F03DF800280AD00649C4
:1006700010310868029A10430860091D0868039A3F
:10068000104308607FBD00000006004030B50F4CED
:10069000002200BF04EB0213D3F800582DB9D3F8A1
:1006A000045815B9D3F808581DB1521C082AF1D3C3
:1006B00030BD082AFCD204EB0212C2F80008C3F8CD
:1006C00004180220C3F8080830BD000000E0014013
:1006D0004FF08050D0F83001082801D0002070473A
:1006E000012070474FF08050D0F83011062905D016
:1006F000D0F83001401C01D0002070470120704725
:100700004FF08050D0F830010A2801D00020704707
:100710000120704708208F490968095808471020B0
:100720008C4909680958084714208A4909680958FA
:100730000847182087490968095808473020854923
:100740000968095808473820824909680958084744
:100750003C20804909680958084740207D490968BC
:100760000958084744207B49096809580847482028
:1007700078490968095808474C207649096809589A
:10078000084750207349096809580847542071499F
:1007900009680958084758206E49096809580847E8
:1007A0005C206C4909680958084760206949096854
:1007B00009580847642067490968095808476820AC
:1007C00064490968095808476C2062490968095852
:1007D000084770205F4909680958084774205D4937
:1007E00009680958084778205A490968095808478C
:1007F0007C205849096809580847802055490968EC
:10080000095808478420534909680958084788202F
:1008100050490968095808478C204E490968095809
:10082000084790204B4909680958084794204949CE
:10083000096809580847982046490968095808472F
:100840009C204449096809580847A0204149096883
:1008500009580847A4203F49096809580847A820B3
:100860003C49096809580847AC203A4909680958C1
:100870000847B0203749096809580847B420354966
:10088000096809580847B8203249096809580847D3
:10089000BC203049096809580847C0202D4909681B
:1008A00009580847C4202B49096809580847C82037
:1008B0002849096809580847CC2026490968095879
:1008C0000847D0202349096809580847D4202149FE
:1008D000096809580847D8201E4909680958084777
:1008E000DC201C49096809580847E02019490968B3
:1008F00009580847E4201749096809580847E820BB
:100900001449096809580847EC2012490968095830
:100910000847F0200F49096809580847F4200D4995
:10092000096809580847F8200A490968095808471A
:10093000FC2008490968095808475FF48070054998
:10094000096809580847000003480449024A034B54
:100950007047000000000020000B0000000B0000AA
:1009600040EA010310B59B070FD1042A0DD310C82C
:1009700008C9121F9C42F8D020BA19BA884201D97E
:10098000012010BD4FF0FF3010BD1AB1D30703D0C6
:10099000521C07E0002010BD10F8013B11F8014B7C
:1009A0001B1B07D110F8013B11F8014B1B1B01D198
:1009B000921EF1D1184610BD02F0FF0343EA032254
:1009C00042EA024200F005B87047704770474FF0A6
:1009D00000020429C0F0128010F0030C00F01B800C
:1009E000CCF1040CBCF1020F18BF00F8012BA8BF1A
:1009F00020F8022BA1EB0C0100F00DB85FEAC17CDE
:100A000024BF00F8012B00F8012B48BF00F8012B90
:100A100070474FF0000200B51346944696462039C1
:100A200022BFA0E80C50A0E80C50B1F12001BFF4A7
:100A3000F7AF090728BFA0E80C5048BF0CC05DF80D
:100A400004EB890028BF40F8042B08BF704748BF5B
:100A500020F8022B11F0804F18BF00F8012B7047CF
:100A6000014B1B68DB6818470000002009480A4951
:100A70007047FFF7FBFFFFF745FB00BD20BFFDE719
:100A8000064B1847064A1060016881F308884068E1
:100A900000470000000B0000000B000017040000DE
:100AA000000000201EF0040F0CBFEFF30881EFF3ED
:100AB0000981886902380078182803D100E0000015
:100AC000074A1047074A12682C3212681047000084
:100AD00000B5054B1B68054A9B58984700BD0000B0
:100AE0007703000000000020F00A0000040000006E
:100AF000001000000000000000FFFFFF0090D00386
:10100000B813002065520200F1C00000CB5102006D
:10101000F1C00000F1C00000F1C0000000000000BD
:10102000000000000000000000000000F15202007B
:10103000F1C0000000000000F1C00000F1C000009D
:10104000595302005F530200F1C00000F1C00000DC
:10105000F1C00000F1C00000F1C00000F1C00000CC
:1010600065530200F1C00000F1C000006B530200A4
:10107000F1C0000071530200775302007D5302005B
:10108000F1C00000F1C00000F1C00000F1C000009C
:10109000F1C00000F1C00000F1C00000F1C000008C
:1010A000F1C0000083530200F1C00000F1C0000055
:1010B000F1C00000F1C00000F1C00000F1C000006C
:1010C00089530200F1C00000F1C00000F1C000002F
:1010D000F1C00000F1C00000F1C00000F1C000004C
:1010E000F1C00000F1C00000F1C00000F1C000003C
:1010F000F1C00000F1C00000F1C00000F1C000002C
:10110000F1C00000F1C0000000F002F824F099F8EE
:101110000AA090E8000C82448344AAF10107DA4552
:1011200001D124F08EF8AFF2090EBAE80F0013F0E7
:10113000010F18BFFB1A43F00103184730470200A4
:10114000504702000A444FF0000C10F8013B13F026
:10115000070408BF10F8014B1D1108BF10F8015B10
:10116000641E05D010F8016B641E01F8016BF9D103
:1011700013F0080F1EBF10F8014BAD1C0C1B09D15A
:101180006D1E58BF01F801CBFAD505E014F8016BCC
:1011900001F8016B6D1EF9D59142D6D3704700005E
:1011A0000023002400250026103A28BF78C1FBD870
:1011B000520728BF30C148BF0B6070471FB500F011
:1011C00003F88DE80F001FBD24F038B870B51A4C35
:1011D00005460A202070A01C00F0D5F85920A080F8
:1011E00029462046BDE8704008F08EB908F097B94E
:1011F00070B50C461149097829B1A0F160015E294A
:1012000008D3012013E0602804D0692802D043F2FB
:1012100001000CE020CC0A4E94E80E0006EB8000A2
:10122000A0F58050241FD0F8806E2846B04720607B
:1012300070BD012070470000080000201800002049
:10124000D45302003249884201D201207047002065
:10125000704770B50446A0F500002E4EB0F1786FCF
:1012600002D23444A4F500042948844201D2012565
:1012700000E0002500F043F848B125B9B44204D39A
:101280002548006808E0012070BD002070BD002DD9
:10129000F9D1B442F9D321488442F6D2F3E710B52C
:1012A0000446A0F50000B0F1786F03D21948044459
:1012B000A4F5000400F023F84FF0804130B1164847
:1012C000006804E08C4204D2012003E01348844209
:1012D000F8D2002080F0010010BD10B520B1FFF75A
:1012E000DEFF08B1012010BD002010BD10B520B1F7
:1012F000FFF7AFFF08B1012010BD002010BD084866
:1013000008490068884201D10120704700207047D9
:1013100000600200000000201C00002008000020E7
:1013200058000020BEBAFECA10B5044600210120B4
:1013300000F041F800210B2000F03DF800210820CA
:1013400000F039F80421192000F035F804210D20AF
:1013500000F031F804210E2000F02DF804210F20B8
:1013600000F029F80421C84300F025F806211620D2
:1013700000F021F80621152000F01DF82046FFF7A7
:1013800025FF002010BDCB2101807047FFF72EBF45
:101390001148704710487047104A10B514680F4B39
:1013A0000F4A08331A60FFF723FF0C48001D046042
:1013B00010BD704770474907090E002804DB00F193
:1013C000E02080F80014704700F00F0000F1E020EA
:1013D00080F8141D7047000003F900421005024018
:1013E00001000001FD48002101604160018170475A
:1013F0002DE9FF4F93B09B46209F160004460DD069
:101400001046FFF726FF18B1102017B0BDE8F08F87
:101410003146012001F0D3FE0028F6D101258DF8D8
:1014200042504FF4C050ADF84000002210A92846A9
:1014300006F0CCFC0028E8D18DF84250A8464FF4C5
:1014400028500025ADF840001C2229466846079523
:101450000CF0D3FF9DF81C000DF11C0A20F00F00CA
:10146000401C20F0F00010308DF81C0020788DF822
:101470001D0061789DF81E000DF1400961F34200E6
:1014800040F001008DF81E009DF8000008AA40F011
:1014900002008DF800002089ADF83000ADF8325020
:1014A0006089ADF83400CDF82CA060680E900AA9D0
:1014B000CDF82890684606F07EFA0028A5D160682D
:1014C000FFF70BFF40B16068FFF710FF20B96078AD
:1014D00000F00300022801D0012000E00020BF4CF2
:1014E00008AA0AA92072BDF8200020808DF8428049
:1014F00042F60120ADF840009DF81E0020F00600E5
:10150000801C20F001008DF81E000220ADF8300094
:10151000ADF8340014A80E90684606F04CFA002886
:1015200089D1BDF82000608036B1211D304600F021
:101530005FF90028C2D109E0BBF1000F05D00CF023
:10154000D7FCE8BB0CF0D4FCD0BBA58017B1012FB1
:1015500043D04AE08DF8428042F6A620ADF8400024
:1015600046461C220021684607950CF046FF9DF870
:101570001C00ADF8346020F00F00401C20F0F0009B
:1015800010308DF81C009DF81D0020F0FF008DF834
:101590001D009DF81E0020F0060040F00100801C98
:1015A0008DF81E009DF800008DF8446040F00200A8
:1015B0008DF80000CDE90A9AADF8306011A800E07E
:1015C00011E00E9008AA0AA9684606F0F4F900286E
:1015D000A6D1BDF82000E08008E00CF089FC10B92D
:1015E0000CF086FC08B103200FE7E58000200CE733
:1015F0003EB50446794D0820ADF80000A88828B112
:101600002046FFF726FE18B110203EBD06203EBD45
:101610002146012001F0D3FD0028F8D12088ADF843
:1016200004006088ADF80600A088ADF80800E088E6
:10163000ADF80A00A88801AB6A46002106F0C2FD99
:10164000BDF800100829E2D003203EBD7FB5634DF0
:101650000446A88868B1002002900820ADF8080070
:10166000CDF80CD02046FFF7F4FD20B1102004B0D7
:1016700070BD0620FBE7A98802AA4FF6FF7006F0AE
:10168000E3FF0028F3D1BDF80810082901D003209A
:10169000EDE7BDF800102180BDF802106180BDF8B3
:1016A0000410A180BDF80610E180E0E701B582B02A
:1016B0000220ADF80000494802AB6A46408800218C
:1016C00006F080FDBDF80010022900D003200EBDF9
:1016D0001CB5002100910221ADF800100190FFF728
:1016E000DEFD08B110201CBD3C486A4641884FF61B
:1016F000FF7006F0A9FFBDF800100229F3D0032007
:101700001CBDFEB5354C06461546207A0F46C0076F
:1017100005D00846FFF79DFD18B11020FEBD0F2033
:10172000FEBDF82D01D90C20FEBD3046FFF791FD1E
:1017300018BB208801A905F040FE0028F4D13078BC
:101740008DF80500208801A906F01AFD0028EBD1CC
:1017500000909DF800009DF8051040F002008DF803
:101760000000090703D040F008008DF80000208831
:10177000694606F0A2FC0028D6D1ADF808502088B2
:101780003B4602AA002106F01DFDBDF80810A94243
:10179000CAD00320FEBD7CB5054600200090019014
:1017A0000888ADF800000C4628460195FFF795FD26
:1017B00018B92046FFF773FD08B110207CBD15B1A4
:1017C000BDF8000060B105486A4601884FF6FF7019
:1017D00006F03AFFBDF8001021807CBD28020020F1
:1017E0000C20FAE72F48C088002800D0012070475D
:1017F00030B5044693B000200D46014600901422F7
:1018000001A80CF0FAFD1C22002108A80CF0F5FD3F
:101810009DF80000CDF808D020F00F00401C20F00B
:10182000F00010308DF800009DF8010006AA20F0AD
:10183000FF008DF801009DF8200001A940F0020092
:101840008DF8200001208DF8460042F60420ADF806
:10185000440011A801902088ADF83C006088ADF8E4
:101860003E00A088ADF84000E088ADF842009DF849
:10187000020020F00600801C20F001008DF802001C
:101880000820ADF80C00ADF810000FA8059008A8CE
:1018900006F091F8002803D1BDF818002880002038
:1018A00013B030BD28020020F0B5007B059F1E4616
:1018B00014460D46012800D0FFDF0C2030803A206E
:1018C0003880002C08D0287A032806D0287B0128ED
:1018D00000D0FFDF17206081F0BDA889FBE72DE96C
:1018E000F04786B0144691F80C900E9A0D46B9F167
:1018F000010F0BD01021007B2E8A8846052807D0C7
:10190000062833D0FFDF06B0BDE8F0870221F2E7FA
:10191000E8890C2100EB400001EB400018803320E7
:101920001080002CEFD0E889608100271AE0009633
:10193000688808F1020301AA696900F086FF06EBD6
:101940000800801C07EB470186B204EB4102BDF89A
:10195000040090810DF1060140460E3212F0C6FEE1
:101960007F1CBFB26089B842E1D8CCE73420108038
:10197000E889B9F1010F11D0122148430E301880C7
:10198000002CC0D0E88960814846B9F1010F00D031
:101990000220207300270DF1040A1FE00621ECE766
:1019A0000096688808F1020301AA696900F04DFFFA
:1019B00006EB0800801C86B2B9F1010F12D007EBCC
:1019C000C70004EB4000BDF80410C18110220AF1E9
:1019D000020110300CF0E7FC7F1CBFB26089B842F6
:1019E000DED890E707EB470104EB4102BDF80400A5
:1019F000D0810AF102014046103212F077FEEBE787
:101A00002DE9F0470E4688B090F80CC096F80C808F
:101A1000378AF5890C20109902F10C044FF0000A66
:101A2000BCF1030F08D0BCF1040F3FD0BCF1070F8D
:101A30007ED0FFDF08B067E705EB850C00EB4C00BC
:101A4000188031200880002AF4D0A8F1060000F0A8
:101A5000FF09558126E01622002101A80CF0CDFCDB
:101A600000977088434601AA716900F0EEFEBDF848
:101A700004002080BDF80600E080BDF80800208149
:101A8000A21C0DF10A01484612F030FEB9F1000F18
:101A900000D018B184F804A0A4F802A007EB080055
:101AA00087B20A346D1EADB2D5D2C3E705EB850C03
:101AB00000EB4C00188032200880002ABAD0A8F130
:101AC000050000F0FF09558137E000977088434614
:101AD00001AA716900F0B9FE9DF80600BDF8041076
:101AE000E1802179420860F3000162F3410182083C
:101AF00062F38201C20862F3C301020962F30411B6
:101B0000420962F34511820962F386112171C0090D
:101B10006071BDF80700208122460DF10901484699
:101B200012F0E4FD18B184F802A0A4F800A000E0CF
:101B300007E007EB080087B20A346D1EADB2C4D2CD
:101B400078E7A8F1020084B205FB08F000F10E0C62
:101B5000A3F800C035230B80002AA6D055819481BC
:101B6000009783B270880E32716900F06EFE61E7F3
:101B70002DE9F84F1E460A9D0C4681462AB1607A2F
:101B800000F58070D080E089108199F80C000C2756
:101B90004FF000084FF00E0A0D2872D2DFE800F077
:101BA0009D070E1B272F374554697272720021461C
:101BB00048460095FFF778FEBDE8F88F207B9146F8
:101BC000082802D0032800D0FFDF3780302009E04A
:101BD000A9F80A80F0E7207B9146042800D0FFDFB7
:101BE000378031202880B9F1000FF1D1E4E7207B64
:101BF0009146042800D0FFDF37803220F2E7207BB7
:101C00009146022800D0FFDF37803320EAE7207BAF
:101C10001746022800D0FFDF3420A6F800A0288055
:101C2000002FC9D0A7F80A80C6E7207B17460428F2
:101C300000D0FFDF3520A6F800A02880002FBBD001
:101C40004046A7F80A8012E0207B1746052802D0FC
:101C5000062800D0FFDF1020308036202880002F9B
:101C6000AAD0E0897881A7F80E80B9F80E00B88173
:101C7000A2E7207B9146072800D0FFDF378037207E
:101C8000B0E72AE04FF0120018804FF0380017003C
:101C9000288091D0E0897881A7F80E80A7F810807D
:101CA00099F80C000A2805D00B2809D00C280DD073
:101CB000FFDF81E7207B0A2800D0FFDF01200AE058
:101CC000207B0B2800D0FFDF042004E0207B0C28C1
:101CD00000D0FFDF052038736EE7FFDF6CE770B5DB
:101CE0000C46054601F0AFFB20B10078222804D253
:101CF000082070BD43F2020070BD0521284610F097
:101D00005DFF206008B1002070BD032070BD30B4BD
:101D10004880087820F00F00C01C20F0F0009030C0
:101D200001F8080B1DCA81E81D0030BC07F06DBC2E
:101D30002DE9FF4784B00027824602970798904616
:101D4000894612300AF025FA401D20F00306079854
:101D500028B907A95046FFF7C2FF002854D1B9F1AE
:101D6000000F05D00798017B19BB052504681BE00F
:101D700098F80000092803D00D2812D0FFDF46E0B4
:101D8000079903254868B0B3497B42887143914263
:101D900039D98AB2B3B2011D10F083FD0446078021
:101DA00002E0079C042508340CB1208810B1032DF3
:101DB00029D02CE00798012112300AF01CFAADF866
:101DC0000C00024602AB2946504608F0A4FA070070
:101DD00001D1A01C029007983A461230C8F80400BE
:101DE000A8F802A003A94046029B0AF011FAD8B154
:101DF0000A2817D200E006E0DFE800F00709141413
:101E0000100B0D141412132014E6002012E61120FA
:101E100010E608200EE643F203000BE6072009E671
:101E20000D2007E6032005E6BDF80C002346CDE9AA
:101E300000702A465046079900F017FD57B9032D48
:101E400008D10798B3B2417B406871438AB2011D43
:101E500010F03BFDB9F1000FD7D0079981F80C9035
:101E6000D3E72DE9FE4F91461A881C468A468046E4
:101E7000FAB102AB494608F04EFA050019D04046C7
:101E8000A61C278810F0DFFF3246072629463B466E
:101E9000009610F0ECFB20882346CDE900504A461E
:101EA0005146404600F0E1FC002020800120BDE8C2
:101EB000FE8F0020FBE710B586B01C46AAB10423B4
:101EC0008DF800301388ADF808305288ADF80A203C
:101ED0008A788DF80E200988ADF80C1000236A4628
:101EE0002146FFF725FF06B010BD1020FBE770B5B7
:101EF0000D46052110F062FE040000D1FFDF2946E7
:101F000004F11200BDE870400AF05EB92DE9F84313
:101F10000D468046002607F075FB044628781028F9
:101F200078D2DFE800F0773B345331311231313170
:101F30000831313131312879001FC0B2022801D077
:101F4000102810D114BBFFDF35E004B9FFDF0521F5
:101F5000404610F033FE007B032806D004280BD047
:101F6000072828D0FFDF072655E02879801FC0B258
:101F7000022820D050B1F6E72879401FC0B20228CD
:101F800019D0102817D0EEE704B9FFDF13E004B929
:101F9000FFDF287901280ED1172137E005214046BF
:101FA00010F00CFE070000D1FFDF07F112014046E0
:101FB0000AF0E7F82CB12A4621464046FFF7A7FE73
:101FC00029E01321404602F01DFD24E004B9FFDFA3
:101FD0000521404610F0F2FD060000D1FFDF694602
:101FE00006F112000AF0D7F8060000D0FFDFA9883A
:101FF000172901D2172200E00A46BDF800008242EC
:1020000002D9014602E005E01729C5D3404600F099
:102010003CFCD0E7FFDF3046BDE8F883401D20F0F0
:10202000030219B102FB01F0001D00E00020104482
:10203000704713B5009848B10024684610F0DBFBE8
:10204000002C02D1F74A009911601CBD0124002028
:10205000F4E72DE9F0470C461546242200212046DE
:102060000CF0CBF905B9FFDFA87860732888DFF89A
:10207000B4A3401D20F00301AF788946DAF80000D0
:1020800010F0D7FB060000D1FFDF4FF000082660FC
:10209000A6F8008077B109FB07F1091D0AD0DAF82C
:1020A000000010F0C6FB060000D1FFDF6660C6F836
:1020B000008001E0C4F80480298804F11200BDE822
:1020C000F0470AF04FB82DE9F047804601F11200C1
:1020D0000D4681460AF05DF8401DD24F20F0030204
:1020E0006E7B14462968386810F0CEFB3EB104FBC5
:1020F00006F2121D03D06968386810F0C5FB052090
:1021000010F004FD0446052010F008FD201A0128F7
:1021100002D1386810F082FB49464046BDE8F047DE
:102120000AF036B870B50546052110F047FD0400E9
:1021300000D1FFDF04F112012846BDE870400AF02B
:1021400020B82DE9F04F91B04FF0000BADF834B04E
:10215000ADF804B047880C4605469246052138463E
:1021600010F02CFD060000D1FFDF24B1A780A4F8F9
:1021700006B0A4F808B0297809220B20B2EB111F91
:102180007ED12A7A04F1100138274FF00C084FF065
:1021900001090391102A74D2DFE802F073F3F2F11F
:1021A0008008D3898EA03DDCF4EFB7B7307B0228DE
:1021B00000D0FFDFA88908EBC001ADF80410302182
:1021C000ADF83410002C25D06081B5F80E900027B2
:1021D0001DE004EBC708317C88F80E10F189A8F8DF
:1021E0000C10CDF800906888042304AA296900F037
:1021F0002CFBBDF81010A8F8101009F10400BDF870
:1022000012107F1C1FFA80F9A8F81210BFB2608963
:10221000B842DED80EE1307B022800D0FFDFE9892A
:1022200008EBC100ADF804003020ADF83400287B85
:102230000A90001FC0B20F90002CEBD06181B5F85E
:102240001090002726E000BFCDF8009068886969EB
:1022500003AA0A9B00F0F9FA0A9804EBC70848445D
:102260001FFA80F908F10C0204A90F9812F03EFA47
:1022700018B188F80EB0A8F80CB0BDF80C1001E049
:10228000D4E0D1E0A8F81010BDF80E107F1CA8F81B
:102290001210BFB26089B842D6D8CBE00DA800902A
:1022A00001AB224629463046FFF719FBC2E0307BDE
:1022B000082805D0FFDF03E0307B082800D0FFDFCF
:1022C000E8891030ADF804003620ADF83400002C59
:1022D0003FD0A9896181F189A18127E0307B09285C
:1022E00000D0FFDFA88900F10C01ADF80410372100
:1022F000ADF83410002C2CD06081E8890090AB89B7
:10230000688804F10C02296956E0E8893921103007
:1023100080B2ADF80400ADF83410002C74D0A98957
:102320006181287A0E280AD002212173E989E1818E
:10233000288A0090EB8968886969039A3CE001214A
:10234000F3E70DA8009001AB224629463046FFF77F
:1023500057FB6FE0307B0A2800D0FFDF1220ADF87A
:102360000400ADF834704CB3A9896181A4F810B0B1
:10237000A4F80EB084F80C905CE020E002E031E0BC
:1023800039E042E0307B0B2800D0FFDF288AADF82F
:1023900034701230ADF8040084B104212173A9898E
:1023A0006181E989E181298A2182688A00902B8AEA
:1023B000688804F11202696900F047FA3AE0307B5C
:1023C0000C2800D0FFDF1220ADF80400ADF8347007
:1023D0003CB305212173A4F80AB0A4F80EB0A4F808
:1023E00010B027E00DA8009001AB224629463046E8
:1023F000FFF75AFA1EE00DA8009001AB22462946CD
:102400003046FFF7B5FB15E034E03B21ADF80400A2
:10241000ADF8341074B3A4F80690A4F808B084F8AA
:102420000AB007E010000020FFDF03E0297A01294D
:1024300017D0FFDFBDF80400AAF800006CB1BDF8AA
:1024400034002080BDF804006080BDF834003928D5
:1024500003D03C2801D086F80CB011B00020BDE8B4
:10246000F08F3C21ADF80400ADF8341014B1697A56
:10247000A172DFE7AAF80000EFE72DE9F8435688DC
:102480000F46804615460521304610F097FB0400A4
:1024900000D1FFDF123400943B46414630466A6863
:1024A00009F0EAFFB8E570B50D46052110F086FB8E
:1024B000040000D1FFDF294604F11200BDE870409E
:1024C00009F074BE70B50D46052110F077FB0400CD
:1024D00000D1FFDF294604F11200BDE8704009F089
:1024E00092BE70B50546052110F068FB040000D1CE
:1024F000FFDF04F1080321462846BDE870400422AE
:10250000AFE470B50546052110F058FB040000D17A
:10251000FFDF214628462368BDE870400522A0E47D
:1025200070B50646052110F049FB040000D1FFDF1D
:1025300004F1120009F02DFE401D20F0030511E00A
:10254000011D00880322431821463046FFF789FC0D
:1025500000280BD0607BABB2684382B26068011D7B
:1025600010F0E9F9606841880029E9D170BD70B5C3
:102570000E46054607F046F8040000D1FFDF0120B3
:10258000207266726580207820F00F00C01C20F059
:10259000F00030302070BDE8704007F036B82DE90B
:1025A000F0438BB00D461446814606A9FFF797FB12
:1025B000002814D14FF6FF7601274FF420588CB134
:1025C00003208DF800001020ADF8100007A805903A
:1025D00007AA204604A912F0A8F878B107200BB08A
:1025E000BDE8F0830820ADF808508DF80E708DF826
:1025F0000000ADF80A60ADF80C800CE00698A178F8
:1026000001742188C1818DF80E70ADF80850ADF8C5
:102610000C80ADF80A606A4602214846069BFFF727
:1026200087FBDCE708B501228DF8022042F60202A2
:10263000ADF800200A4603236946FFF73CFC08BDBD
:1026400008B501228DF8022042F60302ADF8002001
:102650000A4604236946FFF72EFC08BD00B587B083
:1026600079B102228DF800200A88ADF80820498847
:10267000ADF80A1000236A460521FFF759FB07B0A1
:1026800000BD1020FBE709B1072314E407207047C1
:1026900070B588B00D461446064606A9FFF71FFB25
:1026A00000280ED17CB10620ADF808508DF800004E
:1026B000ADF80A40069B6A460821DC813046FFF7E8
:1026C00037FB08B070BD05208DF80000ADF808504C
:1026D000F0E700B587B059B107238DF80030ADF8A9
:1026E0000820039100236A460921FFF721FBC6E772
:1026F0001020C4E770B588B00C460646002506A930
:10270000FFF7EDFA0028DCD106980121123009F01C
:1027100072FD9CB12178062921D2DFE801F0200565
:1027200005160318801E80B2C01EE28880B20AB16E
:10273000A3681BB1824203D90C20C2E71020C0E776
:10274000042904D0A08850B901E00620B9E7012986
:1027500013D0022905D004291CD005292AD007202E
:10276000AFE709208DF800006088ADF80800E08828
:10277000ADF80A00A068039023E00A208DF800005D
:102780006088ADF80800E088ADF80A00A0680A2566
:10279000039016E00B208DF800006088ADF808006B
:1027A000A088ADF80A00E088ADF80C00A0680B2501
:1027B000049006E00C208DF8000060788DF8080089
:1027C0000C256A4629463046069BFFF7B1FA78E7A2
:1027D00000B587B00D228DF80020ADF80810002359
:1027E0006A461946FFF7A4FA49E700B587B071B108
:1027F00002228DF800200A88ADF808204988ADF83B
:102800000A1000236A460621FFF792FA37E71020E4
:1028100035E770B586B0064601200D46ADF80810C4
:102820008DF80000014600236A463046FFF780FA23
:10283000040008D12946304605F0DEFC0021304670
:1028400005F0F8FC204606B070BDF8B51C461546EC
:102850000E46069F10F0E5FA2346FF1DBCB2314636
:102860002A4600940FF0CFFEF8BD30B41146DDE9E2
:1028700002423CB1032903D0002330BC08F029BE3A
:102880000123FAE71A8030BC704770B50C46054644
:10289000FFF72DFB2146284605F0BDFC2846BDE884
:1028A0007040012105F0C6BC4FF0E0224FF400401B
:1028B0000021C2F88001BFF34F8FBFF36F8F17481D
:1028C000016001601649900208607047134900B525
:1028D00000220A600A60124B4FF060721A600028F2
:1028E00008BF00BD0F4A104BDFF840C001280CD0D4
:1028F00002281CBFFFDF00BD032008601A604FF4F0
:10290000000000BFCCF8000000BD022008601A6083
:102910004FF04070F6E700B5FFDF00BD00F5004066
:1029200008F50140A802002014F5004004F501401C
:1029300070B50B2000F0BDF9082000F0BAF90021B5
:102940000B2000F0D4F90021082000F0D0F9F44C5D
:1029500001256560A5600020C4F84001C4F8440169
:10296000C4F848010B2000F0B5F9082000F0B2F9D6
:102970000B2000F091F9256070BD10B50B2000F020
:1029800098F9082000F095F9E5480121416081603F
:10299000E4490A68002AFCD10021C0F84011C0F8BF
:1029A0004411C0F848110B2000F094F9BDE8104024
:1029B000082000F08FB910B50B2000F08BF9BDE8AE
:1029C0001040082000F086B900B530B1012806D0CB
:1029D000022806D0FFDF002000BDD34800BDD34849
:1029E00000BDD248001D00BD70B5D1494FF0004078
:1029F0000860D04DC00BC5F80803CF480024046020
:102A0000C5F840410820C43500F053F9C5F83C41F1
:102A1000CA48047070BD08B5C14A002128B1012818
:102A200011D002281CD0FFDF08BD4FF48030C2F85F
:102A30000803C2F84803BB483C300160C2F84011AB
:102A4000BDE80840D0E74FF40030C2F80803C2F8F0
:102A50004803B44840300160C2F84411B3480CE068
:102A60004FF48020C2F80803C2F84803AD48443050
:102A70000160C2F84811AD48001D0068009008BD13
:102A800070B516460D460446022800D9FFDF002225
:102A9000A348012304F110018B4000EB8401C1F82D
:102AA000405526B1C1F84021C0F8043303E0C0F816
:102AB0000833C1F84021C0F8443370BD2DE9F0411E
:102AC0001D46144630B1012833D0022838D0FFDF2C
:102AD000BDE8F081891E002221F07F411046FFF7FA
:102AE000CFFF012D23D00020944D924F0126687016
:102AF0003E61914900203C3908600220091D0860B0
:102B00008D490420303908608B483D34046008202A
:102B10006C6000F0DFF83004C7F80403082000F010
:102B2000BBF88349F007091F08602E70D0E7012029
:102B3000DAE7012B02D00022012005E00122FBE7A9
:102B4000012B04D000220220BDE8F04198E70122C9
:102B5000F9E774480068704770B500F0D8F8704C19
:102B60000546D4F840010026012809D1D4F808030D
:102B7000C00305D54FF48030C4F80803C4F84061A1
:102B8000D4F8440101280CD1D4F80803800308D5F7
:102B90004FF40030C4F80803C4F84461012012F077
:102BA0008BFDD4F8480101280CD1D4F80803400368
:102BB00008D54FF48020C4F80803C4F84861022007
:102BC00012F07AFD5E48056070BD70B500F09FF8A8
:102BD0005A4D0446287850B1FFF706FF687818B1BF
:102BE0000020687012F068FD5548046070BD032035
:102BF000F8E74FF0E0214FF40010C1F800027047F1
:102C0000152000F067B84B4901200861082000F04A
:102C100061B848494FF47C10C1F80803002002460F
:102C200001EB8003C3F84025C3F84021401CC0B22B
:102C30000628F5D37047410A43F609525143C0F3C1
:102C4000080010FB02F000F5807001EB5020704787
:102C500010B5430B48F2376463431B0C5C020C60F5
:102C6000384C03FB0400384B4CF2F72443435B0D14
:102C700013FB04F404EB402000F580704012107048
:102C800008681844086010BD2C48406870472949FE
:102C90000120C1F800027047002809DB00F01F0284
:102CA000012191404009800000F1E020C0F80011AE
:102CB000704700280DDB00F01F0201219140400900
:102CC000800000F1E020C0F88011BFF34F8FBFF308
:102CD0006F8F7047002809DB00F01F02012191402F
:102CE0004009800000F1E020C0F8801270474907D9
:102CF000090E002804DB00F1E02080F80014704782
:102D000000F00F0000F1E02080F8141D70470C481F
:102D1000001F00680A4A0D49121D1160704700002B
:102D200000B0004004B500404081004044B1004084
:102D300008F5014000800040408500403800002038
:102D400014050240F7C2FFFF6F0C010001000001F3
:102D50000A4810B50468094909480831086012F0AA
:102D60003FFD0648001D046010BD064900200860B4
:102D70004FF0E0210220C1F88002704710050240A8
:102D800001000001FC1F0040374901200860704726
:102D900070B50D2000F049F8344C0020C4F8000153
:102DA0000125C4F804530D2000F050F825604FF0C1
:102DB000E0216014C1F8000170BD10B50D2000F0D5
:102DC00034F82A48012141600021C0F80011BDE813
:102DD00010400D2000F03AB8254810B50468244989
:102DE0002448083108602149D1F80001012804D0A5
:102DF000FFDF1F48001D046010BD1B48001D006858
:102E00000022C0B2C1F8002113F0A3F9F1E710B518
:102E1000164800BFD0F800110029FBD0FFF7DCFFF7
:102E2000BDE810400D2000F011B800280DDB00F0C7
:102E30001F02012191404009800000F1E020C0F80C
:102E40008011BFF34F8FBFF36F8F7047002809DBEE
:102E500000F01F02012191404009800000F1E020B4
:102E6000C0F880127047000004D5004000D0004038
:102E700010050240010000014FF0E0214FF000700A
:102E8000C1F8800101F5C071BFF34F8FBFF36F8FA1
:102E9000C1F80001394B802283F8002441F8800CEE
:102EA000704700B502460420354903E001EBC0033A
:102EB0001B792BB1401EC0B2F8D2FFDFFF2000BD4E
:102EC00041F8302001EBC00100224A718A710122D1
:102ED0000A7100BD2A4A002102EBC000017170474F
:102EE00010B50446042800D3FFDF254800EBC404D6
:102EF0002079012800D0FFDF6079A179401CC0B2A1
:102F0000814200D060714FF0E0214FF00070C1F8B5
:102F1000000210BD70B50425194E1A4C16E0217838
:102F200006EBC1000279012A08D1427983799A42DD
:102F300004D04279827156F8310080472078401CD5
:102F4000C0B22070042801D3002020706D1EEDB2A5
:102F5000E5D270BD0C4810B504680B490B48083128
:102F60000860064890F800044009042800D0FFDFFC
:102F7000FFF7D0FF0448001D046010BD19E000E019
:102F8000E00500205400002010050240010000016F
:102F90000548064A0168914201D1002101600449B7
:102FA000012008607047000058000020BEBAFECA29
:102FB00040E5014070B50C46054609F0F9FB214695
:102FC0002846BDE870400AF0DABC002A14BF4FF46E
:102FD00029614FF4A471002B14BF4FF429624FF400
:102FE000A47200280CBF0120002011449831002851
:102FF00018BF0420084470477047704770470000AE
:103000002CFFFFFFDBE5B15100600200CB00FFFFAA
:1030100084000000C1CF6A00FEA0D9111C1006C3B5
:1030200089CCFC7A7B3B49141906A8C030B5F84D11
:103030000446062CA9780ED2DFE804F0030E0E0E2B
:103040000509FFDF08E0022906D0FFDF04E00329BD
:1030500002D0FFDF00E0FFDFAC7030BD30B50446CA
:103060001038EB4D07280CD2DFE800F0040C060CFA
:103070000C0C0C00FFDF05E0287E112802D0FFDFDA
:1030800000E0FFDF2C7630BD2DE9F04111F0B8FCF7
:10309000044612F0EBFE201AC5B206200FF036FDF2
:1030A000044606200FF03AFD211AD94C207E122842
:1030B00018D000200F1807200FF028FD0646072023
:1030C0000FF02CFD301A3918207E13280CD0002068
:1030D0000144A078042809D000200844281AC0B26E
:1030E000BDE8F0810120E5E70120F1E70120F4E7E8
:1030F000C74810B590F825004108C54800F12600E2
:1031000005D00DF017FEBDE8104006F09DB80DF09B
:10311000F2FDF8E730B50446A1F120000D460A287B
:103120004AD2DFE800F005070C1C2328353A3F445B
:10313000FFDF42E0207820283FD1FFDF3DE0B448A8
:103140008178052939D0007E122836D020782428AD
:1031500033D0252831D023282FD0FFDF2DE0207851
:1031600022282AD0232828D8FFDF26E0207822280A
:1031700023D0FFDF21E0207822281ED024281CD075
:1031800026281AD0272818D0292816D0FFDF14E0C7
:103190002078252811D0FFDF0FE0207825280CD0DB
:1031A000FFDF0AE02078252807D0FFDF05E0207840
:1031B000282802D0FFDF00E0FFDF257030BD1FB5FB
:1031C00004466A46002001F09DFEB4B1BDF802201D
:1031D0004FF6FF700621824201D1ADF80210BDF812
:1031E0000420824201D1ADF80410BDF808108142DC
:1031F00003D14FF44860ADF8080068460EF07EF940
:1032000006F022F804B010BD70B514460D4606460F
:10321000FEF71FF858B90DB1A54201D90C2070BDB9
:10322000002408E056F82400FEF713F808B1102037
:1032300070BD641CE4B2AC42F4D3002070BD2DE933
:10324000F04105461F4690460E4600240068FEF7F2
:103250004DF830B9A98828680844401EFEF746F8A2
:1032600008B110203CE728680028A88802D0B8429E
:1032700002D850E00028F5D0092031E72968085D20
:10328000B8B1671CCA5D152A2ED03CDC152A3AD28B
:10329000DFE802F03912222228282A2A313139396E
:1032A00039393939393939392200085D30BB641C64
:1032B000A4B2A242F9D833E00228DDD1A01C085CF8
:1032C00088F80000072801D2400701D40A2007E748
:1032D000307840F0010015E0C143C90707E001283C
:1032E00007D010E00620FBE60107A1F1805100297C
:1032F000F5D01846F4E63078810701D50B20EFE6CB
:1033000040F0020030702868005D384484B2A8881C
:10331000A04202D2B0E74FF4485382B2A242ADD8E5
:103320000020DDE610B5027843F2022354080122A2
:10333000022C12D003DC3CB1012C16D106E0032C88
:1033400010D07F2C11D112E0002011E080790324ED
:10335000B4EB901F09D10A700BE08079B2EB901F9B
:1033600003D1F8E780798009F5D0184610BDFF2019
:103370000870002010BD08B500208DF8000024481A
:1033800090F82E1049B190F82F0002280ED0032893
:103390000ED0FFDF9DF8000008BD1D4869462530AE
:1033A00001F0FFFD0028F5D0FFDFF3E7032000E088
:1033B00001208DF80000EDE738B50C46054669465A
:1033C00001F0EFFD00280DD19DF80010207861F389
:1033D0004700207055F8010FC4F80100A888A4F830
:1033E0000500002038BD38B51378A8B1022813D0E5
:1033F000FF281AD007A46D46246800944C7905EB89
:103400009414247864F347031370032809D00FE061
:10341000F40100200302FF0123F0FE0313700228D1
:10342000F3D1D8B240F0010005E043F0FE00107087
:10343000107820F0010010700868C2F80100888838
:10344000A2F8050038BD02210FF0B8BB38B50C4614
:103450000978222901D2082038BDADF800008DF886
:10346000022068460DF0A8FC05F0EEFE050003D131
:1034700021212046FFF74EFE284638BD1CB500200E
:103480008DF80000CDF80100ADF80500FE4890F879
:103490002E00022801D0012000E000208DF8070056
:1034A00068460DF00FFD002800D0FFDF1CBD002294
:1034B0000A80437892B263F3451222F040020A80F8
:1034C00000780C282BD2DFE800F02A06090E11162E
:1034D000191C1F220C2742F0110009E042F01D00C8
:1034E00008800020704742F0110012E042F0100006
:1034F00040F00200F4E742F01000F1E742F0010072
:10350000EEE742F0010004E042F00200E8E742F09A
:10351000020040F00400E3E742F00400E0E7072087
:1035200070472DE9FF478AB00025BDF82C60824620
:103530001C4690468DF81C50700703D56068FDF757
:1035400088FE68B9D04F4FF0010997F82E0058B1A6
:1035500097F82F00022807D16068FDF7C7FE18B161
:1035600010200EB0BDE8F087300702D5A089802872
:1035700016D8700705D4B8F1000F02D097F82400D0
:1035800070B1E07DC0F300108DF81B00617D072055
:1035900041B1012906D00229E3D00429E1D12CE070
:1035A0000720DEE749468DF81790F00609D4A27D82
:1035B000072032B1012A04D0022A05D0042AD0D132
:1035C0001BE08DF8191002E002208DF819008DF82B
:1035D00015806068B0B107A9FFF7A4FE0028C0D12C
:1035E0009DF81C00FF280AD0606850F8011FCDF834
:1035F0000F108088ADF8130008E00620B1E743F211
:103600000220AEE7CDF80F50ADF81350E07B002854
:10361000F3D1207C0028F0D1607C0028EDD1A07C83
:103620000028EAD1E07CC006E7D18DF800A0BDF803
:103630002C00ADF80200A0680190A068029004F18F
:103640000F0001F0A2FC8DF80C00FFF794FE8DF83E
:103650000D009DF81C008DF80E008DF816508DF8A9
:103660001850E07D08A900F00F008DF81A00684698
:103670000EF08CF805F0E8FD73E7F0B58FB000258B
:103680008DF830508DF814508DF8345006468DF872
:103690002850019502950395049519B10FC901AC05
:1036A00084E80F00784CA078052801D004280CD1BC
:1036B00001986168884200D120B90398E168884286
:1036C00003D110B108200FB0F0BD207DC00601D598
:1036D0001F2700E0FF273B460DAA05A903A8FFF717
:1036E000AEFD0028EFD1A08AC10702D0C00600D4E9
:1036F000EE273B460AAA0CA901A8FFF7A0FD002867
:10370000E1D19DF81400C00701D00A20DBE7A08AB0
:10371000410708D4A17D31B19DF82810890702D056
:1037200043F20120CFE79DF82810C90709D04007D0
:1037300007D4208818B144F25061884201D907208B
:10374000C1E78DF818508DF81960BDF80800ADF884
:103750001A000198079006A80EF024F805F074FDF1
:103760000028B0D18DF820508DF82160BDF81000F0
:10377000ADF822000398099008A80EF035F805F07E
:1037800063FD00289FD101AD241D95E80F0084E85A
:103790000F00002097E770B586B00D46040005D0F5
:1037A000FDF7A4FD20B1102006B070BD0820FBE796
:1037B0002078C107A98802D0FF2902D303E01F297E
:1037C00001D20920F0E780073BD4FFF75DFC38B158
:1037D0002178C1F3C100012804D0032802D005E0FC
:1037E0001320E1E7284890F82400C8B1C8074FF03B
:1037F00001064FF0000502D08DF80F6001E08DF852
:103800000F50FFF7B8FD8DF8000020786946C0F32F
:10381000C1008DF8010060788DF80250C20801D017
:103820000720C1E778B1C20701D08DF80260820796
:1038300005D59DF8022042F002028DF802204007D3
:1038400003D50620B0E78DF80260002022780B181F
:10385000C2F38002DA7001EB40026388D380401C1F
:10386000A388C0B253810228F0D3207A0028E8D17F
:10387000607A0028E5D1A07A0028E2D1E07A002819
:10388000DFD1207BC00601E0F4010020D9D104F192
:10389000080001F07AFB8DF80E0068460DF0DFFBA2
:1038A00005F0D2FC00288DD18DF810608DF81150F4
:1038B000E088ADF81200ADF8145004A80DF022FC19
:1038C00005F0C2FC00288CD12078C00701D015205B
:1038D00000E01320FFF7C2FB002065E72DE9FF475A
:1038E0000220FD4E8DF804000027708EADF8060012
:1038F000B84643F202094CE001A80FF0C6F80500F3
:1039000006D0708EA8B3A6F83280ADF806803EE0EF
:10391000039CA07F01072DD504F124000090A28E06
:10392000BDF80800214604F1360301F0C5FC05008E
:1039300005D04D452AD0112D3CD0FFDF3AE0A07FC5
:1039400020F00801E07F420862F3C711A1778108E7
:1039500061F30000E07794F8210000F01F0084F884
:1039600020002078282826D129212046FFF7D2FBE5
:1039700021E014E040070AD5BDF8080004F10E016B
:1039800001F019FB05000DD04D4510D100257F1C1D
:10399000FFB202200FF0BAF8401CB842ACD8052D97
:1039A00011D008E0A07F20F00400A07703E0112DE3
:1039B00000D0FFDF0025BDF806007086052D04D07D
:1039C000284604B0CEE5A6F832800020F9E770B5AD
:1039D0000646FFF738FD054605F014FE040000D149
:1039E000FFDF6680207820F00F00801C20F0F000C0
:1039F000203020700320207295F83E006072BDE8F0
:103A0000704005F002BE2DE9F04786B0040000D1F9
:103A1000FFDF2078B04D20F00F00801C20F0F00078
:103A20007030207060680178491F1B2933D2DFE8AD
:103A300001F0FC32323255FB320EFBFB42FA3232DD
:103A40003278FAFAF9F832FAFAF7F6FAFA00C68892
:103A50003046FFF7F8FC0546304607F030FCE0B191
:103A60006068007A85F83E0021212846FFF752FB66
:103A70003046FEF757FB304603F0E2FE31460120A8
:103A800012F02CFEA87F20F01000A877FFF726FF89
:103A9000002800D0FFDF06B064E5207820F0F000B9
:103AA000203020700320207266806068007A607287
:103AB00005F0ABFDD8E7C5882846FFF7C4FC00B980
:103AC000FFDF60680079012800D0FFDF6068017ABD
:103AD00006B02846BDE8F04707F0D6BDC688304698
:103AE000FFF7B1FC050000D1FFDF05F08EFD606837
:103AF00031460089288160684089688160688089D2
:103B0000A881012012F0EAFD0020A875A87F00F02E
:103B100003000228BFD1FFF7E1FE0028BBD0FFDF82
:103B2000B9E7007928B10228B5D03C28B3D0FFDF2F
:103B3000B1E705F06AFD6668B6F806A0307A361D72
:103B4000012806D0687E814605F0EAFA070003D115
:103B500001E0E878F7E7FFDF0022022150460FF08E
:103B600024F8040000D1FFDF22212046FFF7D2FA1B
:103B70003079012800D00220A17F804668F301013E
:103B8000A177308B2081708B6081B08BA08184F80D
:103B900022908DF80880B8680090F86801906A4615
:103BA000032150460FF001F800B9FFDFB888ADF8E7
:103BB0001000B8788DF8120004AA052150460EF0C6
:103BC000F4FF00B9FFDFB888ADF80C00F8788DF885
:103BD0000E0003AA042150460EF0E7FF00B9FFDFF4
:103BE000062106F1120001F004FA40B37079800753
:103BF00000D5FFDF7179E07D61F34700E075D6F80D
:103C00000600A0617089A083062106F10C0001F076
:103C1000F0F9F0B195F825004108607806E043E03E
:103C20003BE072E05AE04FE031E045E061F34700ED
:103C30006070D5F82600C4F80200688D12E0E07DBF
:103C400020F0FE00801CE075D6F81200A061F08A1A
:103C5000D9E7607820F0FE00801C6070F068C4F83E
:103C60000200308AE080B8F1010F04D0B8F1020FF1
:103C700005D0FFDF0FE70320FFF7D8F90BE7287E19
:103C8000122800D0FFDF1120FFF7E8F903E706B0A4
:103C90002046BDE8F04701F09BBD05F0B6FC15F8E5
:103CA000300F40F0020005E005F0AFFC15F8300FD2
:103CB00040F004002870EEE6287E132809D015286D
:103CC000D8D11620FFF7CAF906B0BDE8F04705F0D5
:103CD0009CBC1420F6E70000F4010020A978052917
:103CE00009D00429C6D105F090FC022006B0BDE839
:103CF000F047FFF79BB900790028BBD0E87801F0C6
:103D00002BF905F082FC0320F0E7287E122802D16F
:103D1000687E01F021F91120D4E72DE9F05F054616
:103D200000784FF000080009DFF8B4A891460C466F
:103D3000464601286ED002286DD007280BD00A28ED
:103D40006AD0FFDFA9F8006014B1A4F80080668093
:103D50000020BDE8F09F6968012704F108000B7896
:103D60004FF0020B5B1F4FF6FF721B2B7ED2DFE87A
:103D700003F0647D7D7D0E7D7D7D7D7D7D217D7D5E
:103D80007D2BFDFCFBFA7D14D2F9E7F8F700C8881B
:103D90004FF01208102621469AE14FF01C080A261F
:103DA000BCB38888A0806868807920726868C07910
:103DB0006072C7E74FF01B08142654B3032020722B
:103DC00068688088A080BDE70A793C2ABAD00D1DBA
:103DD0004FF010082C26E4B16988A180298B6182FC
:103DE000298B2182698BA182A98BE1826B790246A2
:103DF000A91D1846FFF7F7FA2979002001290CD0F0
:103E000084F80FB0FF212176E06120626062A06239
:103E100098E70FE03BE15EE199E1E77320760AF174
:103E2000040090E80E00DAF81000C4E90930C4E993
:103E3000071287E7A9F800608AE72C264FF01D08D3
:103E4000002CF7D0A28005460F1D897B008861F306
:103E500000002880B97A490861F341002880B97AC6
:103E6000890861F382002880B97A00E00CE1C90872
:103E700061F3C3002880B97AAA1C0911491C61F3B7
:103E8000041000F07F0028807878B91CFFF7ABFAA7
:103E9000387D05F1090207F11501FFF7A4FA387B17
:103EA00001F0B6F82874787B01F0B2F86874F87EF7
:103EB000A874787AE874387F2875B87B6875388A72
:103EC000E882DAF81C10A961B97A504697F808A080
:103ED000C1F34111012904D0008C504503D2824620
:103EE00009E0FFDF10E0022903D0288820F06000FD
:103EF00009E0504504D1288820F06000403002E0FD
:103F0000288840F060002880A4F824A0524607F1D9
:103F10001D01A8699BE011264FF02008002C89D0D4
:103F2000A280686804F10A02007920726868007B48
:103F3000607269688B1D48791946FFF754FA01E7EA
:103F40000A264FF02108002CE9D08888A0806868F4
:103F5000807920726868C07960729AF8301006E043
:103F600078E06BE052E07FE019E003E03AE021F016
:103F70000401A6E00B264FF02208002CCFD0C88801
:103F8000A0806868007920726868007A01F040F8C3
:103F900060726868407A01F03BF8A072D2E61C2695
:103FA0004FF02608002CBAD0A28068684079607271
:103FB0006868007AA0720AF1040090E80E00DAF84E
:103FC0001000C4E90530C4E90312686800793C2890
:103FD00003D0432803D0FFDFB4E62772B2E684F8AB
:103FE00008B0AFE610264FF02408002C97D0888840
:103FF000A0806868807920816868807A60816868BC
:104000000089A08168688089E0819BE610264FF0D6
:104010002308002C98D08888A0806868C0882081F8
:1040200068680089608168684089A08168688089C3
:10403000E0819AF8301021F0020142E030264FF082
:104040002508002C9AD0A2806968282249680AF0C5
:10405000AAF977E62A264FF02F08002C8ED0A280EE
:1040600069682222091DF2E714264FF01B08002C74
:1040700084D0A280686800790128B0D02772DAE97C
:104080000710C4E903105DE64A46214660E0287A3D
:10409000012803D0022817D0FFDF53E610264FF087
:1040A0001F08002CA2D06888A080A8892081E889F8
:1040B0006081288AA081688AE0819AF8301021F016
:1040C00001018AF830103DE64FF01208102668888A
:1040D00000F07CFF36E6287AC8B3012838D00228E1
:1040E00036D0032801D0FFDF2CE609264FF0110857
:1040F000002C8FD06F883846FFF7A5F990F822A0E2
:10410000A780687A2072042138460EF069FD0521E7
:1041100038460EF065FD002138460EF061FD0121A4
:1041200038460EF05DFD032138460EF059FD0221A0
:1041300038460EF055FD062138460EF051FD072198
:1041400038460EF04DFD504600F006FFFAE5FFE759
:104150002846BDE8F05F01F0C5BC70B5012803D06A
:10416000052800D0FFDF70BD8DB22846FFF76BF940
:10417000040000D1FFDF20782128F4D005F042FAB6
:1041800080B1017821F00F01891C21F0F00110317C
:1041900001700221017245800020A075BDE87040C9
:1041A00005F033BA21462846BDE870401322FFF7D8
:1041B0004DB92DE9F04116460C00804600D1FFDFD5
:1041C000307820F00F00801C20F0F00010303070AC
:1041D0002078012804D0022818D0FFDFBDE8F08144
:1041E0004046FFF730F9050000D1FFDF0320A87536
:1041F00005F00BFA94E80F00083686E80F00F8483F
:1042000010F8301F41F001010170E7E74046FFF769
:104210001AF9050000D1FFDFA1884FF6FF700027D3
:10422000814202D1E288824203D0814201D1E088FA
:1042300040B105F0EAF994E80F00083686E80F006F
:10424000AF75CBE7A87D0128C8D17823002241466D
:1042500012F09AF90220A875C0E738B505460C4659
:104260000846FCF7F6FF70BB232D4AD006DC202D54
:104270000DD0212D23D0222D06D13DE0242D46D076
:10428000252D32D03F2D47D00725284638BD0021A7
:10429000052012F0F9F908B1112038BDA01C0DF06D
:1042A00080F904F0D1FF0500EFD100220823114668
:1042B000052012F069F90528E7D0FFDFE5E760681F
:1042C000FDF70BF808B1102038BD618820886A46D8
:1042D0000DF01BFC04F0B8FF0500D6D16068002883
:1042E000D3D0BDF800100180CFE7A07800F0010125
:1042F00020880DF03BFC17E0206801F09FFE05468A
:10430000C3E7207800F001000CF0E8FC0CE06188C5
:1043100020880DF076FB07E0207800F001008DF892
:10432000000068460CF0A5FF04F08EFFE7E770B5CB
:1043300005460C460846FCF7B2FF08B1102070BDD8
:10434000202D07D0212D0DD0222D0BD0252D09D0C9
:10435000072070BD2088A11C0CF092FDBDE87040C4
:1043600004F072BF062070BD9D482530704708B527
